:100000000EC0189518951895189518951895189567
:1000100018951895189518951895D0C2FBC28FE5BC
:100020008DBFC8E3E9E14E2E81E08EBFD1E0F1E063
:100030005F2EA89584B7082E877F84BF88E1992713
:1000400081BD91BDEEEFF0E0A0E6B0E088278D9392
:100050003197E9F76624B99ABB9ABC9ABD9A80E0B9
:100060008093660080E08093670087E98093680052
:1000700081E08093690080E080936A0086E9809344
:100080006B0080E080936C00E0E0F0E0A0E6B0E080
:1000900092E01AD4E2E0F0E0A2E6B0E092E014D4FC
:1000A0002AD078947FD284EF91E0E6D300918D003E
:1000B000003010F009F001C01BC0759BFECF80918D
:1000C0007E008093610080917F00809360000091AA
:1000D0008D00023010F009F001C008C0809180004E
:1000E0008093630080918100809362005BD203D093
:1000F000DDCFF894FFCFE0E0F0E0A0E6B0E092E0E2
:100100007BE7D1D3E2E0F0E0A2E6B0E092E07BE76B
:10011000CAD302D024D10895C598BC9ABB9AC3987B
:10012000A6E6B0E0119698E08E91983018F4392F39
:10013000992702C038E09850881FC49808F4C49AE0
:1001400000000000C39A00000000C39800000000F7
:100150003A9591F7992341F7BC9ABB9AC398A7E6C1
:10016000B0E0119698E08E91983018F4392F9927C5
:1001700002C038E09850881FC49808F4C49A000060
:100180000000C39A00000000C398000000003A95E8
:1001900091F7992341F7BC9ABB9AC398A8E6B0E0BF
:1001A000119698E08E91983018F4392F992702C053
:1001B00038E09850881FC49808F4C49A00000000E2
:1001C000C39A00000000C398000000003A9591F720
:1001D000992341F7B3D0BC9ABB9AC398AAE6B0E082
:1001E000119698E08E91983018F4392F992702C013
:1001F00038E09850881FC49808F4C49A00000000A2
:10020000C39A00000000C398000000003A9591F7DF
:10021000992341F7BC9ABB9AC398ABE6B0E011961C
:1002200098E08E91983018F4392F992702C038E061
:100230009850881FC49808F4C49A00000000C39A1C
:1002400000000000C398000000003A9591F7992340
:1002500041F7BC9ABB9AC398ACE6B0E0119698E01F
:100260008E91983018F4392F992702C038E09850B1
:10027000881FC49808F4C49A00000000C39A0000C4
:100280000000C398000000003A9591F7992341F7C8
:1002900055D0A0E6B0E00D911C9148E050E0D0D2DE
:1002A000A4E6B0E00D931C93A4E6B0E00D911C9180
:1002B0004DE350E0040F151FA4E6B0E00D931C932E
:1002C000BC9ABB9AC398A4E6B0E0129690E18E91D6
:1002D000983018F4392F992702C038E09850881FB9
:1002E000C49808F4C49A00000000C39A00000000FB
:1002F000C398000000003A9591F7992341F7BC9A02
:10030000BB9AC398A9E6B0E0119698E08E91983018
:1003100018F4392F992702C038E09850881FC498E4
:1003200008F4C49A00000000C39A00000000C398BB
:10033000000000003A9591F7992341F7EF93FF935E
:10034000E4E1F0E090D2FF91EF91C59AEF93FF9333
:10035000E4E1F0E088D2FF91EF91C5980895C1984B
:10036000BC9ABB9AC398A6E6B0E0119698E08E912D
:10037000983018F4392F992702C038E09850881F18
:10038000C49808F4C49A00000000C39A000000005A
:10039000C398000000003A9591F7992341F7BC9A61
:1003A000BB9AC398A7E6B0E0119698E08E9198307A
:1003B00018F4392F992702C038E09850881FC49844
:1003C00008F4C49A00000000C39A00000000C3981B
:1003D000000000003A9591F7992341F7BC9ABB9A27
:1003E000C398A8E6B0E0119698E08E91983018F482
:1003F000392F992702C038E09850881FC49808F414
:10040000C49A00000000C39A00000000C3980000D6
:1004100000003A9591F7992341F7B3D0BC9ABB9A63
:10042000C398AAE6B0E0119698E08E91983018F43F
:10043000392F992702C038E09850881FC49808F4D3
:10044000C49A00000000C39A00000000C398000096
:1004500000003A9591F7992341F7BC9ABB9AC3984B
:10046000ABE6B0E0119698E08E91983018F4392FF1
:10047000992702C038E09850881FC49808F4C49A9D
:1004800000000000C39A00000000C39800000000B4
:100490003A9591F7992341F7BC9ABB9AC398ACE679
:1004A000B0E0119698E08E91983018F4392F992782
:1004B00002C038E09850881FC49808F4C49A00001D
:1004C0000000C39A00000000C398000000003A95A5
:1004D00091F7992341F755D0A2E6B0E00D911C9118
:1004E00048E050E0ADD1A4E6B0E00D931C93A4E643
:1004F000B0E00D911C914DE350E0040F151FA4E6F0
:10050000B0E00D931C93BC9ABB9AC398A4E6B0E0EC
:10051000129690E18E91983018F4392F992702C0E5
:1005200038E09850881FC49808F4C49A000000006E
:10053000C39A00000000C398000000003A9591F7AC
:10054000992341F7BC9ABB9AC398A9E6B0E01196EB
:1005500098E08E91983018F4392F992702C038E02E
:100560009850881FC49808F4C49A00000000C39AE9
:1005700000000000C398000000003A9591F799230D
:1005800041F7EF93FF93E4E1F0E06DD1FF91EF913C
:10059000C19AEF93FF93E4E1F0E065D1FF91EF9111
:1005A000C19808951FD1BA9AB898C29AC09A7FEF9D
:1005B0007FB978EA7DB970EF7EB908950F934F93B4
:1005C0008F939F93AF938FB78F9380E08093930027
:1005D000B898A6E3B0E00C9102FB81E00EF080E059
:1005E0008F93AEE2B0E00C9105FB81E00EF480E069
:1005F0009F918923882309F401C0EBCF78EF7DB95F
:1006000070EF7EB98F918FBFAF919F918F914F9176
:100610000F911895AF920F934F938F93AF938FB71E
:100620008F9300919300003009F018C00FB14EEF86
:100630000423A1E9B0E00C9300919100083609F081
:100640000BC0789B04C081E08093930003C084E0DA
:1006500080939300A0D001C099D090C0033009F0DE
:1006600030C00FB1003009F003C090D087C028C05F
:100670004091900000918F00041709F41BC0009175
:10068000900041E0040FA1E9B0E00C93A1E9B0E0D3
:100690008C918F708C938091910080939000A1E950
:1006A000B0E0AD90BB24ADE6B0E0AA0DBB1D8C91CF
:1006B0008FB902C06BD062C082E08093930077D084
:1006C0005DC0013009F029C04091900000918F0079
:1006D000041709F41BC00091900041E0040FA1E948
:1006E000B0E00C93A1E9B0E08C918F708C93809175
:1006F000910080939000A1E9B0E0AD90BB24ADE6FD
:10070000B0E0AA0DBB1D8C918FB902C03FD036C09E
:1007100082E0809393004BD031C0023009F005C0D5
:1007200083E0809393003DD029C0043009F005C0D8
:1007300085E0809393003FD021C0053009F01EC0B2
:1007400000918D0041E0040FA1E9B0E00C93A1E914
:10075000B0E08C918F708C938091910080938D008C
:10076000A1E9B0E0AD90BB24ADE7B0E0AA0DBB1DA0
:100770008FB18C9384E0809393000DD08F918FBFC5
:10078000AF918F914F910F91AF90189578EA7DB905
:1007900070E77EB9089570E07FB9B89A7EE77EB9B8
:1007A0000895B89870E07FB97EE77EB90895B89A49
:1007B00070E77EB90895B89870E77EB908954091C2
:1007C0008D0000918E00041709F406C0709192000C
:1007D00070687093920005C0709192007F7770935B
:1007E0009200089580E080938E0080E080938D00D9
:1007F00080E08093900080E080938F00089504D083
:100800001FD000FC0CD008950024E89457FF02C0CC
:1008100009D0689400F80BD010F80124089502D094
:1008200009D00895509540954F5F5F4F0895E89423
:1008300017FF0895009510950F5F1F4F6894089556
:10084000752F642F55274427FF93F1E1889405C045
:1008500010F4460F571F5695479517950795FA952B
:10086000B9F7FF9108953197F1F70895689462F808
:100870000895E89462F80895EF93FF93EE27E82B2C
:10088000E92B31F0E0EDF7E03197F1F70197D1F77F
:10089000FF91EF910895E199FECFEEBB3196089557
:1008A00091E001C092E07B3751F47FB7F894F3DF19
:1008B0008D918DBBE29AE19A9A95C9F77FBF772710
:1008C000089591E001C092E0E6DFE09A8DB38D9348
:0608D0009A95D1F708958E
:00000001FF
